:100000000C9438000C9453000C9453000C9453003F
:100010000C947E040C9453000C9453000C945300E5
:100020000C9453000C94E3030C9453000C94530071
:100030000C9453000C9453000C9453000C945300F4
:100040000C940F040C9453000C9453000C9464070C
:100050000C94120E0C9453000C9453000C94530007
:100060000C9453000C9453000C9453000C945300C4
:1000700011241FBECFEFD4E0DEBFCDBF13E0A0E060
:10008000B1E0EAECF7E302C005900D92A633B107A8
:10009000D9F714E0A6E3B3E001C01D92A73BB10776
:1000A000E1F70C945D060C94000090916203292FF7
:1000B000221F2227221F892F82958695869583707D
:1000C0002827892F82958F702827892F86958695D6
:1000D00028272170892F9927880F991F282B209373
:1000E0006203822F99270895FF920F931F93F8942C
:1000F000809138038150823000F180914303863033
:1001000010F0109243038091430380FF02C0949843
:1001100004C0949A88EF0E942F088091430388239B
:1001200039F0809143038F5F80934303789447C3F2
:10013000809143038F5F809343038091370380FF57
:10014000E4C180918D0399278830910541F1893070
:10015000910594F48330910509F48AC084309105A7
:100160001CF4019721F10AC38530910509F41EC1E1
:10017000079709F4A1C002C38B30910509F49CC014
:100180008C30910524F4099709F410C1F7C28D3021
:10019000910509F40BC10F9709F48EC0EFC280E0FE
:1001A0000E94310F80915D030E94FD08E7C280919B
:1001B0004304882321F480913804882361F09091CE
:1001C0005D039F3F41F0991F9927991F8091590323
:1001D000892B0E94310F80913804882309F4CEC204
:1001E00080914004803150F480914004E82FFF2733
:1001F000EB5BFB4F80818F3F09F0C0C2109240043F
:1002000080913F048F5F80933F0480913F04803151
:1002100068F480913F04E82FFF27EE0FFF1FE85E90
:10022000FB4F808191818F5F9F4F11F410923F04AB
:1002300080913F04E82FFF27EE0FFF1FE85EFB4F82
:100240008081918190933B0480933A0480913A0499
:1002500090913B048F5F9F4F21F48FEF8093450473
:100260008DC20E94AD10809353030E94000C86C281
:1002700080914304882309F481C280915D038F3FFC
:1002800029F0881F8827881F0E94310F8091400421
:100290008F5F8093400480914004803150F48091BE
:1002A0004004E82FFF27EB5BFB4F80818F3F09F075
:1002B00065C21092400462C280919604882309F4BA
:1002C0005DC290915D039F3F41F0991F9927991F4F
:1002D00080915903892B0E94310F20915D03822F59
:1002E00099278F739070892B21F080915303820F8F
:1002F00001C0822F0E94FD0880914004803150F49B
:1003000080914004E82FFF27EB5BFB4F80818F3FFC
:1003100009F034C210924004809195048F5F80935D
:10032000950480919504803248F480919504E82FDB
:10033000FF27EB58FB4F80818F3F11F410929504FB
:1003400065E774E085E594E00E943418882331F075
:1003500090915703809156039817A1F0A5E5B4E05A
:10036000E5E7F4E09FE18D918193915097FFFBCFFA
:100370001092950410925303109252030E940B0D99
:100380000E94B40D809156038093570380915203CD
:100390008093530380919504E82FFF27EB58FB4F80
:1003A0006081809157030E94FA14E8C180919604FD
:1003B000882309F4E3C190915D039F3F41F0991FA9
:1003C0009927991F80915903892B0E94310F209101
:1003D0005D03822F99278F739070892B59F01091AC
:1003E0005303120F80913A0490913B040E9498109D
:1003F000810F01C0822F0E94FD088091400480314E
:1004000050F480914004E82FFF27EB5BFB4F808185
:100410008F3F09F0B3C11092400480913F048031B6
:1004200070F480913F04E82FFF27EE0FFF1FE85E76
:10043000FB4F808191818F5F9F4F09F050C01092D8
:100440003F04809195048F5F80939504809195047B
:10045000803248F480919504E82FFF27EB58FB4F3A
:1004600080818F3F59F51092950465E774E085E52A
:1004700094E00E943418882331F0909157038091C2
:100480005603981791F0A5E5B4E0E5E7F4E09FE1A5
:100490008D918193915097FFFBCF1092530310924F
:1004A00052030E940B0D0E94B40D8091560380935D
:1004B0005703809152038093530305C080919504A4
:1004C0008F5F8093950480919504E82FFF27EB5868
:1004D000FB4F6081809157030E94391105C08091C4
:1004E0003F048F5F80933F0480913F04E82FFF27F4
:1004F000EE0FFF1FE85EFB4F8081918190933B04DC
:1005000080933A040E94AD1039C180918D039927E0
:100510008830910541F18930910594F4833091053B
:1005200009F48EC0843091051CF4019771F126C145
:100530008530910509F4BFC0079709F4B2C01EC108
:100540008B30910509F4ADC08C30910524F40997E6
:1005500009F4B1C013C18D30910509F4ACC00F97F7
:1005600009F49FC00BC180915D0380933603809195
:100570005C0380935D030E94550080935C0380912F
:100580005D0340E0642F8F73F3C0809143048823A0
:1005900029F480913804882309F4F0C08091430441
:1005A000882379F080914004803148F480914004A0
:1005B000E82FFF27EB5BFB4F80818F3F11F41092F8
:1005C000400460915D036093360380914004E82FFE
:1005D000FF27EB5BFB4F8F5F80934004E081E0934C
:1005E0005D03EF3F09F4CAC080915803882319F0D6
:1005F000E07CE0935D0320915D03822F99278F7348
:100600009070422F4295469546954370661F662727
:10061000661F2F73892B59F0417080915A03482B24
:1006200080915903682B80915303820F37C041702A
:1006300080915A03482B80915903682B822F2EC03A
:1006400080914304882309F499C00E94000C809192
:1006500040040E94120C80915D03809336038091C8
:100660004004E82FFF27EB5BFB4F808180935D0305
:100670008F3F09F483C00E944B0D20915D03922FA0
:100680009295969596959370917080913603881FF8
:100690008827881F492F682F822F8F730E94160F7B
:1006A0006DC080919604882331F00E94000C8091E7
:1006B00040040E94120C80919604882309F45EC0C5
:1006C00000915D030093360380914004E82FFF27DB
:1006D000EB5BFB4F8F5F80934004E081E0935D0311
:1006E000EF3F09F44BC080915803882319F0E07C58
:1006F000E0935D0320915D03822F99278F739070A3
:10070000422F4295469546954370602F661F662797
:10071000661F2F73892B21F151E0F52EF422809171
:100720005A03F82A00915903062B10915303120F14
:1007300080913A0490913B040E9498104F2D602FB5
:10074000810F0E94160F10915D0380915303180FC3
:1007500080913A0490913B040E949810810F0CC044
:10076000417080915A03482B80915903682B822F46
:100770000E94160F80915D030E94D9088091370373
:10078000843030F485E20E945D0B0E94A60D09C002
:1007900080913703883028F485E20E94BF0B0E94C5
:1007A000990D0E94880D809137038F5F80933703E6
:1007B00080913703883010F01092370378941F919E
:1007C0000F91FF9008951F920F920FB60F92112470
:1007D0002F933F934F935F936F937F938F939F9349
:1007E000AF93BF93EF93FF93809163039091640362
:1007F00090938900809388000E947400FF91EF918C
:10080000BF91AF919F918F917F916F915F914F9128
:100810003F912F910F900FBE0F901F9018951F9230
:100820000F920FB60F9211242F933F934F935F9324
:100830006F937F938F939F93AF93BF93CF93EF93D8
:10084000FF93809144038F3F29F0809144038F5F91
:100850008093440380915403909155038F5F9F4F81
:1008600049F080915403909155030196909355035C
:10087000809354038091410390914203892B81F02E
:10088000809141039091420301979093420380939A
:1008900041038091410390914203892B09F494987C
:1008A000809138038130C1F4C0B3C295CF70C1705C
:1008B00080913E03882371F4CC2361F08091420340
:1008C000909143030196909343038093420388EFF2
:1008D0000E942F08C0933E03FF91EF91CF91BF91EB
:1008E000AF919F918F917F916F915F914F913F91C8
:1008F0002F910F900FBE0F901F9018951F920F927F
:100900000FB60F9211242F933F938F939F9329B388
:10091000237080916503281791F1833041F42230D0
:1009200099F48091600390916103019709C082302E
:1009300059F4233049F4809160039091610301964A
:1009400090936103809360038091600390916103B1
:100950008D52914030F08CE291E09093610380934E
:1009600060038091600390916103449730F484E1C7
:1009700090E09093610380936003209365039F91BF
:100980008F913F912F910F900FBE0F901F90189550
:1009900043E350E081B1886981B940B920E030E09B
:1009A0002CBF4FE150E08AB188698AB949B920BDAE
:1009B00080EC8ABB8CE38BBB8BEB87BB18BA8FEFC9
:1009C00084BB81BB86B981E58DB9089589B7816003
:1009D00089BF8BE083BF8AEF81BF089580917D003E
:1009E000846080937D00089585E20E94BF0B809112
:1009F0007D008B7F80937D000895E199FECF9FBBA2
:100A00008EBBE09A8DB39927089580917D008695DD
:100A100086959927817090700895E199FECF9FBBCC
:100A20008EBB6DBBF894E29AE19A78940895159B79
:100A3000FECF83B980E090E008950F931F93CF938A
:100A4000DF93EC0100E117E2CE01B8010E94AF1B79
:100A50006115710581F0862F805D0E941705CE011A
:100A6000B8010E94AF1BEC01C8016AE070E00E946F
:100A7000AF1B8B010EC0CE01B8010E94AF1BEC0171
:100A8000C8016AE070E00E94AF1B8B016A307105FB
:100A9000D8F601151105A9F0CE01B8010E94AF1BCF
:100AA000CB01805D0E941705CE01B8010E94AF1BEB
:100AB000EC01C8016AE070E00E94AF1B8B01672B5C
:100AC00059F7DF91CF911F910F910895CF93DF9345
:100AD000EC018881882331F089910E941705888173
:100AE0008823D1F7DF91CF9108950F931F93CF9370
:100AF000DF938C0181E00D32180710F00CE211E059
:100B00000431110510F404E110E010935F03009329
:100B10005E03109361030093600360915E0382E0C3
:100B200090E00E940D0580915E0390915F030E940A
:100B30001D0580E091E00E946605C0E0D0E7E8E393
:100B4000F9E3980144275527BE01CF010E94C31B3A
:100B5000FA01E90193E0F695E795D795C7959A953F
:100B6000D1F7BE01CF0126E030E040E050E00E9426
:100B7000C31BFA01E901CA01AA27BB279C01009700
:100B800031F4D0936403C093630381E061C0887F34
:100B9000892B69F403E0F695E795D795C7950A95F3
:100BA000D1F7D0936403C093630382E051C0C901BD
:100BB000807F892B69F414E0F695E795D795C79562
:100BC0001A95D1F7D0936403C093630386E040C0C5
:100BD000C901807E892B69F4B5E0F695E795D79534
:100BE000C795BA95D1F7D0936403C093630387E0A8
:100BF0002FC0C901807C892B69F4A6E0F695E795A2
:100C0000D795C795AA95D1F7D0936403C093630392
:100C100083E01EC0C9018070892B51F48D2F9E2F57
:100C2000AF2FBB27909364038093630384E010C0CD
:100C300020703C7F232B79F46AE0F695E795D795F1
:100C4000C7956A95D1F7D0936403C093630385E099
:100C500080938A0002C010928A0080916303909171
:100C60006403909581959F4F9093640380936303F1
:100C70009093890080938800DF91CF911F910F910D
:100C8000089580916B00816080936B0080916B0070
:100C9000826080936B008BB788608BBF82E090E0AE
:100CA0000E94FD0499270E947505109237038091D8
:100CB0007D00846080937D000895CFEFD4E0DEBF97
:100CC000CDBF0E94C8040E9441060E94E6048091A4
:100CD0005E03809362030E9477090E94B6077894AE
:100CE0000E94C30980918D0399278830910509F4EA
:100CF00084C089309105ECF483309105D1F18430C2
:100D0000910564F48130910509F445C08230910564
:100D10000CF086C0892B09F45EC0E2CF85309105C6
:100D200009F449C0853091050CF45EC0079769F15C
:100D3000D7CF8C30910509F473C08D3091053CF408
:100D40008A30910509F46CC00B9714F53AC08E30C7
:100D5000910531F08E3091053CF10F9799F0C0CF9D
:100D600087E091E00E946605109238030E940B0F05
:100D7000B7CF85E191E00E946605109238030E948A
:100D80008215AECF80E291E011C08BE291E015C0F8
:100D90008EE391E018C082E591E00E946605109212
:100DA00038030E94A6119CCF8EE591E00E94660553
:100DB000109238030DC08AE691E00E94660581E03A
:100DC00005C08EE791E00E94660582E080933803BB
:100DD0000E944D1885CF83E991E00E94660510922C
:100DE00038030E9441087CCF81EA91E00E946605A9
:100DF000109238030E94380F73CF8CEA91E00E9462
:100E00006605109238030E94EE040E94EB0B0E94CC
:100E1000C30980918D038830D1F30E94F40460CF20
:100E20000E94EB0B0E94880D5BCF8F708A3010F40C
:100E3000805D01C0895C0E94170508950895CF93D5
:100E4000DF93EC01892F992782958F70009711F01D
:100E50000E9415078D2F9927009711F00E94150702
:100E6000CE0124E0969587952A95E1F7009711F039
:100E70000E9415078C2F0E941507DF91CF910895CE
:100E800082B1992787FD90958827990F881F992708
:100E90000895179BFECF83B19927089520EA3FE07C
:100EA000E22FF32F3197F1F78A95D1F708958AEF62
:100EB0000E944E078AEF0E944E078AEF0E944E075B
:100EC0008AEF0E944E0708951F920F920FB60F925D
:100ED00011248F939F93EF93FF939CB1983FB1F4AC
:100EE00080913803813021F0949A85E0809341030A
:100EF00080919604882349F18091390390913A03B7
:100F0000019690933A03809339031FC080913C036C
:100F1000E82FFF27E959FC4F90838F5F80933C03B4
:100F200080913C038F7180933C0390913C038091AE
:100F30003D03981751F480913D038F5F80933D03EB
:100F400080913D038F7180933D03FF91EF919F91BD
:100F50008F910F900FBE0F901F90189599270E94A8
:100F6000FD04803108F08FE09927089583E00E9406
:100F7000AE078093870384E00E94AE0780936603E8
:100F8000089590913D0380913C03981719F081E0FA
:100F900090E0089580E090E00895089590913D03D9
:100FA00080913C039817D1F3F89480913D03E82F8A
:100FB000FF27E959FC4F8F5F80933D03908180911B
:100FC0003D038F7180933D037894892F992708956D
:100FD0000E94C107892BC1F00E94CE0787FF14C071
:100FE000682F62956F70482F55276F3059F09A011E
:100FF0002F7030708091870399272817390721F4C3
:1010000060933B03CA01089580E090E0089508953D
:1010100090913603891731F480E00E94310F8FEFF1
:101020008093360308950895CF93C82F962F60E0DC
:10103000992319F40E94080810C0809136038F3F4D
:1010400009F061E08C2F8A51953610F041E001C023
:1010500040E00E94160FC0933603CF9108955D9B28
:10106000FECF8CB980E090E0089580916603806B9C
:101070000E942F088BE70E942F0880E00E942F0813
:1010800008951F93CF930E94F4040E94000C809156
:1010900087030E94120C109194038FEF8093360304
:1010A0000E94C30980918D03882319F00E9435089E
:1010B0007DC00E94570B882339F1412F552780911D
:1010C0009403992701969C01207F3170821B930B1A
:1010D000209187034817590721F4222339F0215022
:1010E00003C02F3019F02F5F20938703609187038F
:1010F00083E090E00E940D050E94000C8091870320
:101100000E94120C109194030E94C107892B41F296
:101110000E94CE07C82F482F441F4427441F89F040
:10112000582F52955F705F3051F099278F709070F3
:101130002091870333278217930709F0B1CF50938B
:101140003B0380913B0399278930910551F08A3008
:1011500091051CF4089789F01CC00E9709F4A0CFE4
:1011600018C0442319F00E94CE07C82F0E94CE0752
:10117000682F8C2F0E94140893CF442319F00E94EB
:10118000CE07C82F0E94CE07682F8C2F0E94080818
:1011900087CF88EB91E00E9466058C2F99270E94EB
:1011A0001F0782ED91E00E9466057ACFCF911F91D3
:1011B0000895CF93C82F8091660380690E942F08FD
:1011C0008C2F99278F739070892B11F480E003C0C6
:1011D0008C2F8F73875E0E942F088C2F82958695A7
:1011E0008695837080FF03C08091B70102C0809113
:1011F000B5010E942F08CF910895CF93C82F8091F9
:10120000660380680E942F088C2F99278F73907037
:10121000892B11F480E003C0CF738C2F875E0E946E
:101220002F088091B6010E942F08CF9108958091D8
:101230003803823029F08CEF0E942F080E94350875
:1012400008950895CF930E940505C82F8091380313
:101250008130D1F0CC2311F00E94F4049498979A35
:1012600085E00E944E0780916303909164030A9782
:101270009093890080938800109243031092370363
:10128000CC2311F00E94EE04CF9108958091380391
:10129000813009F097980895089590B3991F992780
:1012A000991F80914003882339F4992329F0909362
:1012B000400381E090E008959093400380E090E047
:1012C0000895089590B3991F9927991F80913F031E
:1012D000882339F0992329F490933F0381E090E02B
:1012E000089590933F0380E090E00895089581B3BE
:1012F000806F81BB82B38F7082BB08958FE091B302
:10130000982391BB92B3982392BB0895DE980895D9
:10131000AC01F894C0980000000000000000C09AE2
:1013200020E01FB8779BFECFFA01E20FF11D8FB1CD
:1013300080832F5F2330A8F37894089599B396950E
:1013400096959F70292F269526952695892F869507
:101350008270282B892F9927880F991F382F347076
:10136000232B880F991F880F991F8870282B8FE0D7
:10137000821B99270895DE9A089589B386958695EC
:101380008F7099270895AF92BF92CF92DF92EF921C
:10139000FF920F931F93CF93DF93CDB7DEB72697BE
:1013A0000FB6F894DEBF0FBECDBF20916003309121
:1013B000610380915E0390915F032817390731F034
:1013C00080916003909161030E947505A1E9B3E0EB
:1013D000EAE8F3E042E011921D92415047FFFBCF53
:1013E00080914403843108F490C0109244030E9419
:1013F0008609CE0101960E94880980918E038C8314
:1014000080918F038D83809190038E8340E001E073
:1014100010E06E01C00ED11E842F869586958695AC
:10142000A82FBB27BD0162577C4F842F877098017E
:1014300002C0220F331F8A95E2F7C901FB013081F8
:10144000232F2823FD01EB56FC4FE081E823AC0D50
:10145000BD1DAC91A8234F5F8095222331F0382326
:10146000EA2B3E2BDB013C9305C03823EA233E2BBD
:10147000FB013083483180F20E949E09482F809101
:101480009403481749F080918903481729F4409341
:10149000940381E080934503409389030E94BB0934
:1014A00061E9E62E63E0F62E0AE813E06EE873E0E9
:1014B00055E9A52E53E0B52EF60142E08081D50115
:1014C0008D935D012381DB018D91BD01922F9827C2
:1014D0008923D8018D938D019223D7019D937D019E
:1014E0004150319647FFEACF0E94BD09482F8091B5
:1014F0008D03481731F080918803481711F4409309
:101500008D03409388030E94880D26960FB6F894A9
:10151000DEBF0FBECDBFDF91CF911F910F91FF9026
:10152000EF90DF90CF90BF90AF900895282F883133
:1015300018F080E090E00895869586958695E82FCE
:10154000FF27E257FC4F80819927277002C09595AD
:1015500087952A95E2F79C012170307080FF03C0C7
:1015600081E090E00895C90108950895282F8831F9
:1015700018F080E090E00895869586958695E82F8E
:10158000FF27E657FC4F80819927277002C0959569
:1015900087952A95E2F79C012170307080FF03C087
:1015A00081E090E00895C90108950895282F8831B9
:1015B00018F080E090E00895869586958695E82F4E
:1015C000FF27EF56FC4F80819927277002C0959521
:1015D00087952A95E2F79C012170307080FF03C047
:1015E00081E090E00895C9010895089580918E03E7
:1015F000882359F480918F03882339F480919003D4
:10160000882319F481E090E0089580E090E0089547
:101610000895FF920F931F93CF93DF93FF2400E071
:1016200010E0CDEDD1E088810E94960A882311F068
:10163000C80109C0F39421960F5F1F4F8CE08F15EE
:1016400094F78FEF9FEFDF91CF911F910F91FF9054
:101650000895CF93C0E0EC2FFF27EB52FE4F80811F
:101660000E94960AEC2FEF5F882319F08E2F99279E
:1016700005C0CE2FE83078F380E090E0CF91089558
:10168000CF93C0E0EC2FFF27EB52FE4F80810E94EA
:10169000B60AEC2FEF5F882319F08E2F992705C02B
:1016A000CE2FE83078F380E090E0CF9108958091DC
:1016B00045031092450399270895282F883290F406
:1016C000869586958695E82FFF27E55BFC4F27706A
:1016D00081E090E002C0880F991F2A95E2F72081EF
:1016E000282B208308950895282F883290F486951A
:1016F00086958695E82FFF27EA5BFC4F277081E0EF
:1017000090E002C0880F991F2A95E2F72081282BCC
:10171000208308950895282F8832A0F48695869511
:101720008695E82FFF27EA5BFC4F277081E090E069
:1017300002C0880F991F2A95E2F7982F9095808113
:101740008923808308950895282F883218F080E037
:1017500090E00895869586958695E82FFF27EA5BA9
:10176000FC4F277081E090E002C0880F991F2A95F6
:10177000E2F720812823822F992708950895282FA2
:101780008832A0F4869586958695E82FFF27E55B3D
:10179000FC4F277081E090E002C0880F991F2A95C6
:1017A000E2F7982F9095808189238083089508958A
:1017B000282F869586958695EBE4F3E0E80FF11DDA
:1017C00080819927277002C0959587952A95E2F721
:1017D00081709070089510924F0310924E031092F2
:1017E0004D0310924C0310924B0310924A03109237
:1017F000490310924803109247031092460308953C
:101800000F931F93CF9307E112E0CFE0F80181918E
:101810008F010E94BF0BC150C7FFF8CFCF911F911E
:101820000F910895803138F4E82FFF27E95EFD4FCE
:1018300080810E945D0B08950895803138F4E82F6F
:10184000FF27E95EFD4F80810E94740B0895089583
:10185000803118F020E030E009C0E82FFF27E95E72
:10186000FD4F80810E94D80B282F3327C90108958E
:10187000803118F080E090E00895E82FFF27E95EBE
:10188000FD4F80810E94A40B992708950895883107
:1018900038F4E82FFF27E150FE4F80810E945D0B56
:1018A00008950895883138F4E82FFF27E150FE4F5E
:1018B00080810E94740B08950895883138F4E82FD0
:1018C000FF27E150FE4F80810E94BF0B08950895CD
:1018D0000F931F93CF930FEF11E0C7E1F8018191B0
:1018E0008F010E94BF0BC150C7FFF8CFCF911F914E
:1018F0000F910895E82F8150883030F4FF27EA5087
:10190000FE4F80810E945D0B089508951F93CF9331
:10191000182F81E0E82FFF27C82FCF5F811731F400
:10192000EA50FE4F80810E945D0B05C0EA50FE4FD9
:1019300080810E94BF0B8C2FC93060F3CF911F9123
:101940000895E82F8150883030F4FF27EA50FE4F89
:1019500080810E94BF0B08950895E82F8150883040
:1019600030F4FF27EA50FE4F80810E94740B0895E7
:101970000895E82F8150883040F4FF27EA50FE4F49
:1019800080810E94A40B9927089580E090E008953B
:101990000895E82F8150883048F4FF27EA50FE4F21
:1019A00080810E94D80B282F332702C020E030E02E
:1019B000C90108950F931F93CF9307EF11E0C7E07C
:1019C000F80181918F010E94BF0BC150C7FFF8CF72
:1019D000CF911F910F9108958D3038F4E82FFF2794
:1019E000E651FE4F80810E945D0B089508958D3071
:1019F00038F4E82FFF27E651FE4F80810E94740BD8
:101A000008950895EAEEF1E0E80FF11D80810E944B
:101A1000A40B992708950F931F93CF930AEE11E01B
:101A2000CCE0F80181918F010E94BF0BC150C7FF2C
:101A3000F8CFCF911F910F9108950E940B0D84E074
:101A40000E94BF0B83E00E94BF0B88E00E94BF0B87
:101A500081E00E94BF0B82E00E94BF0B0895CF93EC
:101A6000C82F84E00E94BF0BC23021F483E00E94A3
:101A7000740B0FC083E00E94BF0B83E00E948B0BAE
:101A8000C13011F483E003C0CF3F19F484E00E9419
:101A90005D0BCF910895CF93C82F0E941D0DC7FFF6
:101AA00003C086E10E94470C8C2F8295869586950F
:101AB000837080FF03C085E10E94470CCF7311F44F
:101AC0008C2F15C0C73110F48FEF11C0C43218F439
:101AD000CC5080E00CC0C03318F4C85181E007C07E
:101AE000CC3318F4C45282E002C083E0C0530E9499
:101AF0002F0DCC2321F484E10E94470C07C0EC2F6A
:101B0000FF27E152FE4F80810E945D0BCF91089527
:101B1000F894DF98EBE4F3E080818FB9779BFECFF8
:101B2000319683E0EF34F807B9F3B4F3DF9A789491
:101B30000895A6E4B3E0EBE4F3E024E080819D9116
:101B4000892B8193215027FFF9CF0895A6E4B3E0B4
:101B5000EBE4F3E024E09D919095808189238193CB
:101B6000215027FFF8CF0895A6E4B3E0EBE4F3E0BB
:101B700034E020819C91822F892319F090952923AC
:101B800020831D923150319637FFF3CF0895AC0179
:101B900020E0322F6115710581F0FA01E30FF11D8C
:101BA00080812827E22FFF27E95DFD4F20813F5FDD
:101BB000832F99278617970780F3822F99270895F7
:101BC0000F931F93CF93DF936115710549F08C013B
:101BD000EB01F80181918F010E9417052197C9F748
:101BE000DF91CF911F910F9108950F931F9308E9F3
:101BF00013E090E8909398031092990391E09093EA
:101C00009A0380939B0364E070E0C8010E94C70DB3
:101C100080939C0365E070E0C8010E94E00D1F9175
:101C20000F9108951F920F920FB60F921124EF9209
:101C3000FF921F932F933F934F935F936F937F93E5
:101C40008F939F93AF93BF93CF93DF93EF93FF93C4
:101C500093B180912703882309F4C5C08091510373
:101C6000803448F4E82FFF27E852FC4F90838F5FC1
:101C70008093510304C00E94F50D109251032091EE
:101C80005103233008F4AFC0F090D8038091D903FA
:101C9000682F7727762F66278091DA039927682B9C
:101CA000792B3327CB0104962817390708F49BC0FA
:101CB000FB01E852FC4F1381EB012396BE0188ED36
:101CC00093E00E94C70D181791F0BE0188ED93E0D4
:101CD0000E94C70D99270E941F071092510380E0B0
:101CE0000E94F50D0E94000C0E94880D7EC08F2D71
:101CF00099278031910509F44AC08131910524F476
:101D0000019709F469C06AC0419709F067C08091E2
:101D1000DA03823009F062C08091DB039091DC032A
:101D2000C82FDD27CC0FDD1FCC0FDD1FCC0FDD1F33
:101D3000C90FD11D89E1809398031092990380E126
:101D400080939A030F2EFBE9EF2EF3E0FF2EF02D88
:101D500034E0CC0FDD1F3A95E1F71FE0CE010E9481
:101D60005510F70181937F011150219617FFF6CF8F
:101D700063E170E088E993E00E94C70D8093AB03B4
:101D800064E170E088E993E00E94E00D2AC0809150
:101D9000DA03823119F58091DB039091DC03C82FBF
:101DA000DD2723E0CC0FDD1F2A95E1F7C90FD11DF8
:101DB0009DEDE92E93E0F92E84E0CC0FDD1F8A958E
:101DC000E1F71FE0BE01F70181917F010E9416102B
:101DD0001150219617FFF6CF81E001C080E00E94EC
:101DE000F50D109251030E94000CFF91EF91DF91CD
:101DF000CF91BF91AF919F918F917F916F915F91A3
:101E00004F913F912F911F91FF90EF900F900FBE38
:101E10000F901F9018950E94C30980918D038E30FA
:101E2000D1F30E94EB0B0E94880D089590E03A9840
:101E3000803408F08FE3611160E4442311F440E83A
:101E400001C0492F882349F0862B842B85BB3A9A01
:101E50009F5F9832E8F3399A0895642B65BB089523
:101E60000895882311F0AE9A01C039983A980895E0
:101E70007F928F929F92AF92BF92CF92DF92EF921A
:101E8000FF920F931F93CF93DF93EE24FF248824B8
:101E9000982C0E94EE040E94000C7090940367013D
:101EA00057010E94C30980918D03843019F00E946C
:101EB0003508AEC08091660399270E94280C892BB3
:101EC00031F40E94000C809166030E94120C0E9463
:101ED000570B882309F1472D5527809194039927A3
:101EE00001969C01207F3170821B930B2091660329
:101EF0004817590721F4222339F0215003C02F300D
:101F000019F02F5F209366036091660384E090E0F0
:101F10000E940D05709094038E2D0E942F0D00E0FD
:101F2000C8E2D3E088810E94B60A8823A1F0102F6E
:101F30001A0D195E492D682D812F0E94160F892DCB
:101F4000992756E0880F991F5A95E1F7812B0E9437
:101F5000D90841E0842E88810E94D60A882369F03E
:101F6000202F2C0D295E892D992736E0880F991F87
:101F70003A95E1F7822B0E94FD080F5F21960D3004
:101F800088F28FE00E94B60A882351F082E0E816BA
:101F9000F104D4F40894E11CF11C8CE090E010C032
:101FA0008EE00E94B60A882379F09FEFE9169FEF32
:101FB000F90651F04CF00894E108F10884EF9FEF26
:101FC000A80EB91EC80ED91E85E10E94B60A882344
:101FD00071F080E0992009F481E0982E882321F0A7
:101FE00081E00E945D0B03C081E00E94BF0B83B3C0
:101FF00099278F739070892B09F453CF0E94F60AAA
:10200000882309F44ECF80E00E94310F882449CF05
:10201000DF91CF911F910F91FF90EF90DF90CF90C4
:10202000BF90AF909F908F907F900895282FF89445
:1020300095E0C09800000000000000009FB9779B69
:10204000FECF00000000000000001FB8779BFECF0D
:102050008FB1C09A000000000000000080FDE9CFB1
:10206000C0980000000086E08FB9779BFECF00008B
:102070000000C09A0000000000000000C0980000AE
:10208000000082E08FB9779BFECF872F99278FB909
:10209000779BFECF6FB9779BFECF2FB9779BFECF93
:1020A00000000000C09A789408959C01F894C098AC
:1020B0000000000083E08FB9779BFECF832F992724
:1020C0008FB9779BFECF2FB9779BFECF0000000022
:1020D0001FB8779BFECF8FB1C09A78949927089547
:1020E00010923C04109243041092380480E00E9445
:1020F000310F0E94EB0B0E94B40D0E94570B089504
:1021000010923D0484E20E94BF0B0E94EB0B0E94E0
:10211000B40D1092430480E00E94310F089581E0D5
:1021200080933D0484E20E945D0B0E94000C0895A0
:10213000892F9927282F2F71822F992787FD909516
:1021400034E0969587953A95E1F7892B09F0206E52
:10215000822F992787FD9095089520913A04277042
:1021600080913A0490913B04F3E096958795FA9517
:10217000E1F7622F8F700E94FA1460913A04709117
:102180003B049B0144275527DA01C90180709078F0
:10219000A070B070892F9A2FAB2FBB278093580364
:1021A000DA01C90180709074A070B070892F9A2FE5
:1021B000AB2FBB2780935A03207030724070507051
:1021C000BB27A52F942F832F80935903109240048F
:1021D000CB010E9498109927089581E080933C04D8
:1021E00081E20E945D0B10925A0380915A03809302
:1021F0005903809159038093580310923804109228
:102200004304809118049091190490933B048093A7
:102210003A048F5F9F4F89F010923F041092400460
:1022200010925D030E94AD10809353038091370399
:1022300080FDFCCF81E0809338040E94000C08955B
:1022400080915303882321F483E00E94BF0B0CC0CC
:1022500087FF07C083E00E94BF0B84E00E945D0BF4
:10226000089583E00E945D0B84E00E94BF0B0895F7
:102270000895FF920F931F93CF93DF93C82FDD270D
:1022800003E0CC0FDD1F0A95E1F7C60FD11D15E065
:10229000CC0FDD1F1A95E1F7BFE0FB2EC050D84FE1
:1022A00008E114E0CE010E9455109927982F882745
:1022B000F80180839183CE0101960E945510282F4A
:1022C0003327F80180819181822B932B8193919305
:1022D0008F01FA942296F7FEE5CFDF91CF911F91FF
:1022E0000F91FF900895FF920F931F93CF93DF9369
:1022F000C82FDD2753E0CC0FDD1F5A95E1F7C60F3D
:10230000D11D45E0CC0FDD1F4A95E1F73FE0F32EEC
:1023100008E114E0C050D84FF80180819181892FE5
:102320009927BE010E9416102196F8018191919182
:102330008F01BE010E941610FA942196F7FEECCF91
:10234000DF91CF911F910F91FF9008951F93CF932D
:10235000DF930E94EE048091940387708093390488
:1023600010923E0410923D0410923C0410923804E6
:102370001092430410923F048FEF9FEF90933B0421
:1023800080933A04109238030E94000C0E94B40D0E
:102390000E94C30980918D03813071F00E94F40482
:1023A000109243041092380480E00E94310F0E9482
:1023B000EB0B0E94880DF4C280913D04882361F5E7
:1023C00080913C04882341F50E94570B882359F0E3
:1023D0008091940387708093390460913E040E9439
:1023E00039110E94000C809139040E94120C0E9445
:1023F000290BC82F882359F00E940B0D8C2F815078
:1024000080933E04682F809139040E943911809195
:102410003E048F5F0E947A0C81E00E94B60A8823F6
:1024200079F080913C04882319F00E94701008C054
:1024300080913D04882311F00E9480100E94ED10CD
:1024400080913C04882329F480913D04882309F479
:1024500063C080913F040E94380C882311F40E94CD
:10246000B40D80913F040E941D0C80913A0490911C
:102470003B048F5F9F4F21F40E941D0D80E046C0FA
:1024800080E00E94BF0B80913A0490913B0443E0AE
:10249000969587954A95E1F78F700E94120C80916E
:1024A0003A0490913B0497FF04C088E00E945D0BC2
:1024B00003C088E00E94BF0B80913A0490913B04D6
:1024C000AA27BB273EE0B695A795979587953A959D
:1024D000D1F781709070892B21F081E00E945D0B13
:1024E00003C081E00E94BF0B80913A0490913B04AD
:1024F000AA27BB272DE0B695A795979587952A958E
:10250000D1F781709070892B21F082E00E945D0BE1
:1025100003C082E00E94BF0B88E00E94B60A8823B5
:1025200031F483E00E94B60A882309F478C0109140
:102530003C04112309F073C0812F0E94310FC09118
:102540003D04CC2309F442C088E00E94B60A8823E7
:10255000D1F080913F049927019640976CF48091C7
:102560003F04E82FFF27EE0FFF1FE85EFB4F80813F
:1025700091818F5F9F4F19F410933F0430C0809179
:102580003F048F5F20C080913F048823C9F480916D
:102590003F0499270196409714F580913F04E82F56
:1025A000FF27EE0FFF1FE85EFB4F808191818F5F59
:1025B0009F4FA9F080913F048F5F80933F04E7CF46
:1025C00080913F04815080933F0409C088E00E94BD
:1025D000B60A882321F00E948F10C0933F04809197
:1025E0003F04E82FFF27EE0FFF1FE85EFB4F8081BF
:1025F000918190933B0480933A04109243048F5F3F
:102600009F4F69F00E94AD108093530310924004D5
:102610008091370380FDFCCF81E08093430487E104
:102620000E94B60A882339F180913D048823E9F09D
:1026300080913F0499270196409764F480913F046C
:10264000E82FFF27EE0FFF1FE85EFB4F8FEF9FEF96
:10265000828393838FEF9FEF90933B0480933A04A0
:102660000E94801080E00E94BF0B60913E04809128
:1026700039040E94731180913D04882309F47FC1BD
:1026800080913A0490913B048F5F9F4F09F40FC1F2
:1026900084E10E94B60A882311F180913F04E82F5B
:1026A000FF27EE0FFF1FE85EFB4F8081918120E046
:1026B00030E8822793278083918380819181909352
:1026C0003B0480933A04AA27BB2780709078A070BF
:1026D000B070892F9A2FAB2FBB278093580385E1C9
:1026E0000E94B60A882311F180913F04E82FFF274A
:1026F000EE0FFF1FE85EFB4F8081918120E030E408
:1027000082279327808391838081918190933B04DA
:1027100080933A04AA27BB2780709074A070B07091
:10272000892F9A2FAB2FBB2780935A0386E10E94F3
:10273000B60A882311F180913F04E82FFF27EE0F9E
:10274000FF1FE85EFB4F8081918120E030E282270D
:102750009327808391838081918190933B04809320
:102760003A04AA27BB2780709072A070B070892F9E
:102770009A2FAB2FBB27809359038FE00E94960AB4
:10278000882331F48EE00E94960A882309F47DC0E4
:102790000E94090BC82FDD27C7FDD0958FE00E944E
:1027A000B60A882329F48EE00E94B60A882351F0E5
:1027B0000E94B40D0E940B0D83E00E94BF0B84E0C9
:1027C0000E94BF0B8FE00E94960A882349F183E0A4
:1027D0000E945D0B8FEFCF3FD807C9F00E94B40D68
:1027E00020913A0430913B04307E9C2F8827282B7F
:1027F000392B30933B0420933A0480913F04E82F17
:10280000FF27EE0FFF1FE85EFB4F2083318380918F
:102810003A0490913B040E9498108093530332C075
:102820008EE00E94960A882309F441C084E00E9449
:102830005D0B2FEFCF3FD207E1F00E94B40D209146
:102840003A0430913B04307E2C97CF71D0709C2F8E
:102850008827282B392B30933B0420933A0480910E
:102860003F04E82FFF27EE0FFF1FE85EFB4F20839A
:10287000318380913A0490913B040E949810809398
:102880005303845F0E94F70C12C08FE00E94D60AA7
:10289000882329F48EE00E94D60A882341F083E041
:1028A0000E94BF0B84E00E94BF0B0E94B40D8FE01A
:1028B0000E94960A882309F062C08EE00E94960A60
:1028C000882309F05CC00E94400BC82F882329F49C
:1028D0000E94570B882309F447C00E94DA0C0E941B
:1028E000000CCC2359F480913A0490913B048F5F03
:1028F0009F4F29F0C0913A04C77001C0C150109297
:10290000430480E00E94310F40919403242F332729
:1029100063E0220F331F6A95E1F78C2F9927282B4C
:10292000392B30933B0420933A0480913F04E82FE5
:10293000FF27EE0FFF1FE85EFB4F208331836C2FD4
:10294000842F0E94FA14109240041092590380912F
:10295000590380935A0380915A038093580310922D
:10296000530381E0809343040E94201180913A0434
:1029700090913B048770907001960E94860C809124
:102980003C04882309F404CD0E94201180913A046C
:1029900090913B048770907001960E94860CF8CC51
:1029A000DF91CF911F9108951092400481E08093B0
:1029B000410481E20E945D0B80E00E94310F0E9481
:1029C000EE048091370380FDFCCF81E080934304C7
:1029D000089581E080933D0484E20E945D0B0E9493
:1029E000000C80E00E94120C0E94F40480E00E941F
:1029F000310F0895EF92FF920F931F93CF93DF93C0
:102A0000182F062F0E94880DC12FDD2723E0CC0F41
:102A1000DD1F2A95E1F7C00FD11D94E0CC0FDD1F1B
:102A20009A95E1F785E4E82E84E0F82E1FE0CE01C8
:102A30000E945510F70181937F011150219617FFD5
:102A4000F6CF0E94880DDF91CF911F910F91FF90DB
:102A5000EF900895EF92FF920F931F93CF93DF9320
:102A6000182F062F0E94880DC12FDD2753E0CC0FB1
:102A7000DD1F5A95E1F7C00FD11D45E4E42E44E077
:102A8000F42E34E0CC0FDD1F3A95E1F71FE0BE01D4
:102A9000F70181917F010E9416101150219617FFB6
:102AA000F6CF0E94880DDF91CF911F910F91FF907B
:102AB000EF90089510923D0484E20E94BF0B0E94A3
:102AC000680C0E94000C809194030E94120C0E94DA
:102AD000EE0480E00E94310F08950E94F4041092E9
:102AE00043040E94680C0E94000C809194030E9491
:102AF000120C1092410481E20E94BF0B80E00E9400
:102B0000310F0895EF92FF920F931F93CF93DF93AE
:102B10001092420410923D0410924104109243041A
:102B20001092400410925D03109238030E94C30972
:102B30008091940380934404609142040E94FA14AB
:102B40000E94EB0B809194030E94120C0E94EE04F1
:102B50000E94C30980918D03833081F00E94F404A8
:102B60001092430480E00E94310F0E9446090E94A7
:102B700017090E94EB0B0E94880D6FC290914404CC
:102B8000809194039817D1F080914104882311F02B
:102B90000E946D1580913D04882311F00E945A1502
:102BA0008091940380934404609142040E94FA143B
:102BB0000E94000C809194030E94120C80914104A9
:102BC0008823E1F480913D048823C1F4809142047C
:102BD0008F5F0E947A0C0E94290BC82F882371F006
:102BE0000E940B0D8C2F0E947A0C8C2F81508093A9
:102BF0004204682F809144040E94FA1480E00E94ED
:102C0000B60A882399F080914104882379F082E202
:102C10000E945D0B05E414E0CFE00E945500F8012E
:102C200081938F01C150C7FFF8CF0CC080E00E9494
:102C3000D60A882339F080914104882319F082E272
:102C40000E94BF0B81E00E94B60A882379F0809130
:102C50004104882319F00E946D1508C080913D043D
:102C6000882311F00E945A150E94D41480914104C7
:102C7000882329F480913D04882309F427C1009119
:102C80004004E02EFF24E701CB5BDB4F18811F736C
:102C900085E10E94B60A882331F01F3321F0888134
:102CA00090E48927888386E10E94B60A882349F048
:102CB0001F3339F0F701EB5BFB4F808190E88927E8
:102CC00080831F3341F0112331F0173110F4CFEF1F
:102CD0000DC0143210F4C0E009C0103310F4C1E08C
:102CE00005C01C3310F4C2E001C0C3E084E10E94BF
:102CF000B60A811110E08FE00E94B60A882339F0ED
:102D00001F3329F0112319F0C2300CF4145F8EE048
:102D10000E94B60A882341F01F3331F0112321F0BD
:102D2000CF3F11F00CF01C5084E00E94B60A8823BB
:102D300031F08CE0C802C0011124182F195E89E01F
:102D40000E94B60A882331F08CE0C802C001112429
:102D5000182F185E85E00E94B60A882331F08CE0B7
:102D6000C802C0011124182F175E8AE00E94B60A1B
:102D7000882331F08CE0C802C0011124182F165EA0
:102D8000C3300CF063C086E00E94B60A882331F09D
:102D90008CE0C802C0011124182F155E87E00E9444
:102DA000B60A882331F08CE0C802C0011124182F24
:102DB000145E8BE00E94B60A882331F08CE0C802D2
:102DC000C0011124182F135E81E10E94B60A8823E6
:102DD00031F08CE0C802C0011124182F125E8CE083
:102DE0000E94B60A882331F08CE0C802C001112489
:102DF000182F115E82E10E94B60A882331F08CE020
:102E0000C802C0011124182F105E8DE00E94B60A7E
:102E1000882331F08CE0C802C0011124182F1F5DF7
:102E200080E10E94B60A882331F08CE0C802C0011C
:102E30001124182F1E5D83E10E94B60A882331F009
:102E40008CE0C802C0011124182F1D5D202F3327EC
:102E5000F901EB5BFB4F80818F3F11F41F3319F4B5
:102E60008081807C182BE901CB5BDB4F88811817B0
:102E7000F9F080913D04882331F080E00E94310F09
:102E800081E00E944E07188380913D04882381F0E1
:102E9000812F82958695869583708170912F991FD9
:102EA0009927991F482F692F812F8F730E94160F22
:102EB0001F3F39F0812F0E944B0D80E00E94BF0B15
:102EC00005C00E941D0D80E00E945D0B88E00E94FD
:102ED000B60A882331F483E00E94B60A882309F4F5
:102EE0009BC080913D04882309F46AC080E00E9461
:102EF000310F81E00E944E0788E00E94B60A8823C5
:102F0000B1F0809140049927019640974CF480914C
:102F10004004E82FFF27EB5BFB4F80818F3F19F4C4
:102F20001092400420C0809140048F5F1AC08091AD
:102F30004004882399F4809140048F30A0F480915C
:102F40004004E82FFF27EB5BFB4F80818F3F59F058
:102F5000809140048F5F80934004EDCF80914004C6
:102F60008150809340040E94000C809140040E9494
:102F7000120C80914004E82FFF27EB5BFB4F808110
:102F800080935D038F3F51F481E00E94BF0B82E08C
:102F90000E94BF0B80E00E945D0B3EC080E00E945B
:102FA000BF0B80915D03982F92959695969593709F
:102FB0009170282F221F2227221F492F622F25C000
:102FC00088E00E94B60A882339F1C0914104CC23DD
:102FD00019F50E94E914C093400480914004E82F41
:102FE000FF27EB5BFB4FE081E0935D03EF3FA1F038
:102FF0008E2F829586958695837081709E2F991F5E
:103000009927991F482F692F8E2F8F730E94160FB3
:1030100080915D030E944B0D87E10E94B60A8823D0
:1030200009F496CD80913D04882381F0809140047D
:1030300099270196409744F480914004E82FFF2798
:10304000EB5BFB4F8FEF81830E945A156091420426
:10305000809194030E942A157BCDDF91CF911F911F
:103060000F91FF90EF90089540E0DB01FC0190810B
:103070008C91981719F080E090E0089580818F3F3F
:1030800019F481E090E008954F5F31961196403237
:1030900070F381E090E008950895EF92FF920F930E
:1030A0001F93CF93FF24E0908D03809138038823F2
:1030B00019F40E94EE040BC00E94F40480913803BE
:1030C000813019F40E947E0902C00E9477090E9493
:1030D000EB0B0E94B40D10927504809175048093DF
:1030E00055048FEF80937604809176048093560484
:1030F00081E00E947A0C1092960410923F04109284
:10310000400410923B0410923A04109295041092DD
:103110005203109253030E94000C80918D038F3054
:1031200021F08B3011F08730D1F4809194031AC0D4
:10313000109296040E9446090E94170910925203A9
:1031400010925303109259031092580310925A038D
:103150000E94EB0B0E94B40D0E94880DFAC2809170
:103160009403877080935703809356038091940350
:103170000E94120C0E94C30980918D038E15C1F626
:1031800087E10E94B60A882329F180915403909127
:10319000550386509D40D0F480915403909155037F
:1031A0008E54914098F0209154033091550380E65D
:1031B0009AEEB9010E94AF1B7093550360935403BC
:1031C00080915403909155030E9475051092550308
:1031D0001092540380E00E94B60A882349F00E94AE
:1031E0000B0D0E94B40D82E20E945D0B10925B03F6
:1031F00080E00E94D60A882329F1A7E9B4E0E5E53A
:10320000F4E0CFE18D918193C150C7FFFBCF809156
:1032100096048823A1F4A5E5B4E0E5E7F4E0CFE166
:103220008D918193C150C7FFFBCF80915203809352
:10323000530383E00E94BF0B84E00E94BF0B82E235
:103240000E94BF0B80E00E94960A882361F1C0E0D3
:1032500080915B03C81760F4EC2FFF27E956FB4F02
:103260008081883028F48F5F0E947A0CCF5FF0CF86
:103270000E94400BC82F882309F44EC180915B0344
:10328000803208F049C1E82FFF27E956FB4FC150B3
:10329000C0838F5F80935B03E82FFF27E956FB4FC6
:1032A0008FEF808339C18FE00E94960A882331F422
:1032B0008EE00E94960A882309F46DC00E94090BD3
:1032C000C82F8FE00E94B60A882329F48EE00E945E
:1032D000B60A882339F00E940B0D0E94B40D82E2D9
:1032E0000E94BF0B8FE00E94960A882301F184E0C0
:1032F0000E94BF0B83E00E945D0BCF3F11F0C09393
:1033000052038091530387FD0AC00E94020D882357
:1033100031F40E94B40D809153030E94F70C9091F8
:10332000520380915303981761F1892F28C08EE0D2
:103330000E94960A882329F183E00E94BF0B84E053
:103340000E945D0BCF3F19F0CC50C0935203809187
:103350005303181664F0845F0E94020D882339F429
:103360000E94B40D80915303845F0E94F70C9091EA
:10337000520380915303981721F0892F845F0E9494
:10338000EC0C80919604882309F0C6C0809152030A
:1033900080935303C1C08FE00E94D60A882329F48A
:1033A0008EE00E94D60A882321F00E940B0D0E9415
:1033B000B40D0E94290BC82F882331F40E94570BAB
:1033C000882309F446C01FC00E94DA0CC150C09384
:1033D000550480915504809397048FEF8093560491
:1033E000809156048093980480919604882319F55F
:1033F000A5E5B4E0E5E7F4E0CFE18D918193C1501C
:10340000C7FFFBCF18C080918D038F3021F08B3028
:1034100011F0873019F48091940303C080919403D4
:1034200087708093560380919604882321F48091BD
:1034300056038093570380919604882351F40E9489
:10344000000C809156030E94120C809152038093CD
:10345000530365E774E085E594E00E9434188823FF
:10346000F9F4809156048F3F49F4809176048F3FA0
:1034700029F4809175048F5F0E94AD0CC0E005E5D2
:1034800014E0F8018081893008F044C0D8018D91A2
:103490008D018F5F0E947A0CCF5FC03290F33AC0EB
:1034A000C0E005E714E0F8018081893098F580914B
:1034B00096048823E1F080919504E82FFF27EB58CC
:1034C000FB4FD8019C918081981789F48C918F5F74
:1034D0000E94B90C8823C9F4F80180818F5F0E9493
:1034E000A10CD8018C918F5F0E94AD0C0EC0F80129
:1034F00080818F5F0E94B90C882311F00E94B40D67
:10350000D8018C918F5F0E947A0CCF5F0F5F1F4FA5
:10351000C03248F20E94201180919604882351F114
:1035200080913803823089F48091390390913A0375
:1035300018161906FCF48091390390913A03039709
:1035400090933A038093390312C0813099F48091AB
:103550004203909143031816190664F480914203C4
:1035600090914303039790934303809342030E94F7
:10357000740000CE80913803823019F40E94E8076D
:10358000F82E80913803882349F481E00E94B60A1E
:10359000882321F080919604882371F48091380368
:1035A000823021F4BCEFFB1639F02BC0813049F595
:1035B0000E946209882329F11092960480E00E94FB
:1035C000310F0E94170980913803813011F00E9459
:1035D000460981E20E94BF0B0E94B40D0E94000CBC
:1035E00080918D038F3021F08B3011F0873019F4EA
:1035F0008091940303C08091940387700E94120C01
:1036000068C080913803882349F481E00E94B60A9B
:10361000882321F080919604882389F080913803D3
:10362000823029F48F2D8A5F823048F052C0813079
:1036300009F04FC00E944D09882309F44AC081E275
:103640000E945D0B80918D038F3021F08B3011F043
:10365000873039F460917504809194030E94FA14C4
:1036600011C0809194036091750487700E94391194
:10367000809118049091190490933B0480933A042C
:103680000E94AD1010925D0380913803823019F4CE
:10369000EBEFFE1631F01092950410924004109258
:1036A0003F041092370310923A031092390310929C
:1036B0004303109243031092420381E080939604E7
:1036C0008AEF0E942F0880913803813011F00E9408
:1036D000220986E10E94B60A882331F081E08093B6
:1036E000590382E00E945D0B86E10E94D60A88237E
:1036F00029F01092590382E00E94BF0B85E10E94DD
:10370000B60A882329F081E080935A030E945D0B5A
:1037100085E10E94D60A882329F010925A0381E09D
:103720000E94BF0B84E10E94B60A882331F081E039
:103730008093580388E00E945D0B84E10E94D60AC2
:10374000882309F417CD1092580388E00E94BF0B1C
:1037500011CDCF911F910F91FF90EF900895AA1B6B
:10376000BB1B51E107C0AA1FBB1FA617B70710F06C
:10377000A61BB70B881F991F5A95A9F7809590959E
:10378000BC01CD010895A1E21A2EAA1BBB1BFD01AD
:103790000DC0AA1FBB1FEE1FFF1FA217B307E40730
:1037A000F50720F0A21BB30BE40BF50B661F771F88
:1037B000881F991F1A9469F7609570958095909568
:0A37C0009B01AC01BD01CF0108958B
:1037CA002042504D0A0D00436F6D70436F6E747244
:1037DA006F6C0A0D0050617474456469740A0D00B7
:1037EA0050617474506C61790A0D005061747450A0
:1037FA006C61792044494E53594E430A0D00506179
:10380A007474506C6179204D69646953594E430A46
:10381A000D00547261636B456469740A0D00547239
:10382A0061636B506C61790A0D00547261636B506D
:10383A006C61792044494E53594E430A0D00547223
:10384A0061636B506C6179204D49444953796E63C9
:10385A000A0D004D494449436F6E74726F6C0A0D2C
:10386A00004B6579626F6172640A0D0072416E44A1
:10387A00306D0A0D0064207F526563656976656460
:10388A0020556E6B6E6F776E204D4944493A203051
:10389A0078000A0D00040506071112101304090521
:1038AA000A06070B110C120D1013201B191C1A18EB
:1038BA000F0C0E0B0D0A0920191A180C0B0A0922F3
:1038CA0021252320191A18241B1C0F0E0D04030A84
:1038DA000C0B090801020026271D1E1F10121113C6
:1038EA001415161705060700070E091C1B121538B2
:1038FA003F363124232A2D70777E796C6B626548B6
:10390A004F464154535A5DE0E7EEE9FCFBF2F5D825
:10391A00DFD6D1C4C3CACD90979E998C8B8285A8D5
:10392A00AFA6A1B4B3BABDC7C0C9CEDBDCD5D2FF3E
:10393A00F8F1F6E3E4EDEAB7B0B9BEABACA5A28FF5
:10394A0088818693949D9A2720292E3B3C35321FE5
:10395A0018111603040D0A5750595E4B4C45426F15
:10396A0068616673747D7A898E878095929B9CB113
:10397A00B6BFB8ADAAA3A4F9FEF7F0E5E2EBECC135
:10398A00C6CFC8DDDAD3D4696E676075727B7C51A5
:10399A00565F584D4A4344191E171005020B0C2155
:1039AA00262F283D3A33344E49404752555C5B76C0
:1039BA0071787F6A6D64633E39303722252C2B0675
:1039CA0001080F1A1D1413AEA9A0A7B2B5BCBB9665
:1039DA0091989F8A8D8483DED9D0D7C2C5CCCBE695
:1039EA00E1E8EFFAFDF4F3010409050A06070B11F1
:0639FA000C120D10130079
:00000001FF
